:107000000C944C380C9469380C9469380C94693899
:107010000C9469380C9469380C9469380C9469386C
:107020000C9469380C9469380C9469380C94EE3DD2
:107030000C94203E0C9469380C9469380C9469388F
:107040000C9469380C9469380C9469380C9469383C
:107050000C9469380C9469380C9469380C9469382C
:107060000C9469380C9469380C9469380C9469381C
:107070000C9469380C9469380C9469380C9469380C
:107080000C9469380C9469380C9469380C946938FC
:107090000C9469380C94693811241FBECFEFD4E0EA
:1070A000DEBFCDBF11E0A0E0B1E0E6E3FFE702C044
:1070B00005900D92A436B107D9F711E0A4E6B1E02E
:1070C00001C01D92A43CB107E1F70E946B380C94FB
:1070D000993F0C940038DF93CF9300D0CDB7DEB743
:1070E0001A8219820E94E5380E94AD380E945F3FE3
:1070F0000E949C3B81E085BF82E085BF789481E05F
:1071000090E00E94CB382091560180E090E0A0E012
:10711000B0E00FC080E090E0A0E0B0E002C022301C
:10712000D9F4E981FA81E491EF3FA1F30196A11D21
:10713000B11D8C3737EC93073CE0A30730E0B30771
:1071400071F780E090E00E94CB38F8940E94553FA0
:10715000E0E0F0E00995FFCFFFCF14B817B81AB8F8
:1071600015B818B81BB8269A3F9A249A0E944C3931
:10717000479885E0982F9A95F1F7479A8A95F1F705
:107180000E94643983EC0E943A3984E00E943A39C3
:107190000E9443390895009711F02E9A08952E9871
:1071A0000895F89428EC30E02E9A88EE93E0F901E7
:1071B0003197F1F70197D9F72E9888EE93E0F9010E
:1071C0003197F1F70197D9F7EFCF14BE80916000A6
:1071D00080618093600080E18093600080E880930C
:1071E00061001092610080E090E041E2FC013E9677
:1071F00040935700E4919C01220F331F220F331F4D
:10720000D90112965E2F52955F705A3010F4505D7E
:1072100001C0595AA050BF4F5C932C5F3F4FEF7095
:10722000EA3010F4E05D01C0E95AD901A050BF4F27
:10723000EC9301968A309105C9F60895FA01D901B7
:107240008330A1F4662319F0613081F406C08AE22C
:1072500091E09183808384E005C080E091E0918398
:1072600080838AE28C9321E030E002C020E030E0AD
:10727000C90108958093CE008091C80087FFFCCF9C
:107280008091CE000895599A089510926501109248
:1072900064011092C9000895599A559A539A519AC7
:1072A0005298ECECF0E01182108280EC8093CA00DE
:1072B00088E18093C9001182108281E090E0909370
:1072C0006501809364010895809164019091650146
:1072D000009711F40E944C39599808951092660154
:1072E00010926701109268011092690108959C0143
:1072F00040E050E08091660190916701A0916801A3
:10730000B0916901280F391F4A1F5B1F61E070E0CF
:10731000213080E7380780E0480780E0580710F008
:1073200060E070E0CB0108952F923F924F925F9200
:107330006F927F928F929F92AF92BF92CF92DF9285
:10734000EF92FF920F931F93CF93DF93EB01A090E7
:107350006601B0906701C0906801D090690190907B
:107360006A01860175010894E11CF11C011D111DC3
:10737000A6019501DC013C01660E771E93E0892E83
:107380005524539485E0482E44C0CA01B9016F7753
:10739000707080709070611571058105910539F4E8
:1073A000F90180925700E89507B600FCFDCFC901AE
:1073B000817090706C91009769F0892D90E0362E65
:1073C000222482299329F9010C0150925700E89553
:1073D000112401C0962EC801B7016F7770708070BC
:1073E0009070611571058105910549F4F701E05828
:1073F000F04040925700E89507B600FCFDCF11968B
:107400000894E11CF11C011D111D2F5F3F4F4F4FD0
:107410005F4FA615B70509F0B8CFCE01A0E0B0E0E8
:107420008A0D9B1DAC1DBD1D809366019093670165
:10743000A0936801B093690190926A01DF91CF91A6
:107440001F910F91FF90EF90DF90CF90BF90AF9082
:107450009F908F907F906F905F904F903F902F9074
:1074600008958091660190916701A0916801B091A3
:1074700069019C01AD012F7730704070507021156B
:1074800031054105510549F0807825E0FC01209344
:107490005700E89507B600FCFDCF81E180935700C7
:1074A000E8950895EF92FF920F931F93CF93DF9388
:1074B000DC01E0906601F090670100916801109195
:1074C0006901A801970108C0E491ED9361507040F3
:1074D0002F5F3F4F4F4F5F4FF901E901CE19DF0991
:1074E0006115710541F0203080E8380780E04807D9
:1074F00080E0580749F72093660130936701409375
:10750000680150936901CE01DF91CF911F910F91D6
:10751000FF90EF9008950895FC01608171818FE6DE
:1075200091E00E9494390895EF92FF920F931F9378
:10753000CF93DF93EC01398120E0888190E0822BAA
:10754000932B21E081329207A1F0E1E082329E0785
:107550002CF48132910509F0DDC0E1C0F2E0813AFE
:107560009F0709F472C026E08132920709F0D2C069
:10757000CBC080915601823049F48A819B819093DF
:107580006C0180936B010E946E3903C0853009F055
:10759000C9C080915601823059F080916B01909161
:1075A0006C0101972A813B812817390709F4B7C07C
:1075B0002A813B8180916B0190916C0128173907DA
:1075C00009F06AC00E80DF81C02D209761F40E940F
:1075D000313A82E08093560181E090E090936E0111
:1075E00080936D019CC0CE010E947739009711F401
:1075F00088E004C0C134D10530F08EE080935201A0
:1076000020E030E015C0D093B001C093AF0189EB0A
:1076100091E061E070E04FE651E02C2F0CE81AE3B6
:107620003FEAE32E31E0F32E0E94FE3B21E030E002
:1076300080916B0190916C01019690936C01809305
:107640006B0185E0809356016FC0809156018230B6
:1076500049F48A819B8190936C0180936B010E9415
:107660006E3903C0893009F05DC0809156018230C7
:1076700051F080916B0190916C0101972A813B81BF
:107680002817390749F02A813B8180916B0190913D
:107690006C012817390739F08AE0809356018EE093
:1076A000809352013CC00E80DF81C02DC134D105D2
:1076B00020F08EE0809352011AC08FE691E0BE0167
:1076C0000E94523A9C018C179D0720F482E080931F
:1076D000560101C09E0189EB91E062E070E04FE647
:1076E00051E000E010E0EE24FF240E94FE3B809178
:1076F0006B0190916C01019690936C0180936B01EA
:1077000089E0809356010BC082E08093560110926D
:10771000520105C0CE010E94AF3B9C0105C021E093
:1077200030E002C020E030E0C901DF91CF911F912D
:107730000F91FF90EF90089584E99AE39093B80138
:107740008093B7018CEE9BE39093B2018093B101DB
:107750008BE89AE39093B4018093B3010895EF927C
:10776000FF920F931F93FC01318120E0808190E014
:10777000822B932B24E08132920781F025E0813A1D
:10778000920791F023E0813A9207F1F489EB91E0BE
:1077900062E070E042E551E026E00DC082E08093B7
:1077A0005601109252010DC089EB91E062E070E049
:1077B00046E551E021E000E010E0EE24FF240E94C5
:1077C000FE3B21E030E002C020E030E0C9011F9123
:1077D0000F91FF90EF900895813221F00E941E39A1
:1077E0009C010AC088E591E0FA019183808389E0D9
:1077F000F901808321E030E0C90108958F929F92C2
:10780000AF92BF92CF92DF92EF92FF920F931F93AE
:10781000DF93CF930F92CDB7DEB74C015B016A01C6
:10782000FC0180819181009721F029830E94D13849
:107830002981F401B182A082D382C282C20ED11CFE
:10784000D582C48210870783F286E186C4010E9434
:10785000DA3D0F90CF91DF911F910F91FF90EF9044
:10786000DF90CF90BF90AF909F908F900895FF9240
:107870000F931F93DF93CF9300D00F92CDB7DEB756
:10788000DC0111969C91119780E02C9130E0282B1F
:10789000392B83E0233038070CF583E0203038079C
:1078A0000CF02FC1233831054CF4213831050CF090
:1078B00028C12038310509F017C14CC081E02030C3
:1078C000380709F41BC181E0203038070CF40CC1E3
:1078D00081E0233038070CF007C113C188E020385D
:1078E000380709F4ABC088E02138380784F486E013
:1078F0002038380709F452C087E02030380709F4EF
:1079000000C185E02030380709F0EEC042C08AE0AF
:107910002138380709F4F5C08AE02238380734F4F2
:1079200089E02030380709F0DFC0AFC08BE021309C
:10793000380731F08CE02238380709F0D5C0E1C0B3
:107940002091420130E0205C3E4F80E090E0E9E48D
:10795000F1E0C6C016968D919C91179782309105E3
:1079600009F0CFC001E611E08091B9019091BA0110
:10797000009711F00E94D13882E090E09093BA0114
:107980008093B9011093BC010093BB010E5F1F4FA0
:107990006BC012968C910E94C03DB0C012966C9143
:1079A000129713968C91139716960D911C91179719
:1079B000813019F0823099F407C08EE291E09B8308
:1079C0008A8380912E0109C0662309F09AC080E461
:1079D00091E09B838A8380914201898311C0E09169
:1079E000B101F091B201309709F48BC0AE014E5F46
:1079F0005F4F9E012F5F3F4F0995009709F481C0AB
:107A0000898190E00817190708F409830A811B810E
:107A1000F9808091B9019091BA01009711F00E940C
:107A2000D13882E090E09093BA018093B90110932D
:107A3000BC010093BB010F0D111D16C003E611E040
:107A40008091B9019091BA01009711F00E94D1384C
:107A500082E090E09093BA018093B9011093BC0149
:107A60000093BB010F5F1F4F1093BE010093BD0138
:107A70001092C1011092C0011092C3011092C20174
:107A800089EB91E00E94DA3D39C08091450190E098
:107A900021E030E012964D915C91139748175907F9
:107AA00081F531C0628170E014964D915C9115971B
:107AB0006417750789F4638170E012964D915C91AB
:107AC00013976417750741F4E091B501F091B60181
:107AD0003097A1F0099512C001964081E40FF11D85
:107AE000E217F307F9F60DC0E091B701F091B80184
:107AF000309739F0CD0109959C0105C021E030E0B7
:107B000002C020E030E0C9010F900F900F90CF919C
:107B1000DF911F910F91FF900895E1EFF0E0208138
:107B20003081932F80E030E0282B392BC901089554
:107B30008091E80080FFFCCF8091E3008068809313
:107B4000E30008951092E90089E08093EB00109221
:107B5000EC0080E38093ED008091ED0082608093E3
:107B6000ED008091EE0087FFFCCF8FE08093F00066
:107B70001092BA011092B90180E48093BF01089578
:107B8000EF92FF920F931F938093E30089EB91E0B4
:107B900062E070E040E050E020E008E91DE3EE2400
:107BA000FF240E94FE3B81E090E01F910F91FF9027
:107BB000EF900895FC01208131812230310569F474
:107BC000895B914063EA7BE80E94873F8093E900EC
:107BD0008091F00081608093F00008951F920F92D1
:107BE0000FB60F9211242F933F934F935F936F9390
:107BF0007F938F939F93AF93BF93EF93FF93809166
:107C0000E10083FF0CC0E091B301F091B401309723
:107C100009F009950E94A23D87EF8093E100FF9152
:107C2000EF91BF91AF919F918F917F916F915F91F4
:107C30004F913F912F910F900FBE0F901F9018956D
:107C40001F920F920FB60F921124EF92FF920F9393
:107C50001F932F933F934F935F936F937F938F93D4
:107C60009F93AF93BF93EF93FF93DF93CF93CDB7E2
:107C7000DEB72897DEBFCDBF8091F40080FFFBC048
:107C80001092E9008091E80083FF3BC01092BA0196
:107C90001092B9018091F200883010F40E94D1381E
:107CA0008091F10089838091F1008A830E948D3D4B
:107CB0009C838B830E948D3D9E838D830E948D3D8E
:107CC00098878F83CE0101960E94373C009709F474
:107CD000BDC0898187FDC7C08091B9019091BA016B
:107CE000009709F0C0C089EB91E062E070E040E0ED
:107CF00050E020E000E010E0EE24FF240E94FE3B74
:107D0000B2C08091E80082FF4EC08091B90190918D
:107D1000BA018130910509F099C06091F200262FD7
:107D200030E08091BD019091BE014091BB01509126
:107D3000BC01841B950B821793070CF487C008C005
:107D40008091F1008193F093BC01E093BB016150FD
:107D5000E091BB01F091BC01662391F78091BD01D8
:107D60009091BE01E817F90709F081C01092BA019D
:107D70001092B901E091C001F091C101309729F052
:107D80008091C2019091C301099589EB91E062E075
:107D900070E040E050E020E000E010E0EE24FF243E
:107DA0000E94FE3B64C08091E80081FF07C01092F2
:107DB000BA011092B9018DEF8093E8008091E8003C
:107DC00080FF59C08091B9019091BA01823091052C
:107DD000B9F58091BD012091BB019091BF01821B3B
:107DE000981708F4892F982F0CC0E091BB01F091EF
:107DF000BC0121912093F100F093BC01E093BB0101
:107E00009150992391F79091BF01891721F0109219
:107E1000BA011092B9018EEF8093E8008091B90108
:107E20009091BA01009739F5E091C001F091C1013C
:107E3000309709F18091C2019091C30109951BC04F
:107E40008091F0008E7F8093F00015C081EF8093C9
:107E5000E8001092BA011092B9018091EB008062A3
:107E60008093EB0008C087EF8093E8004ACF8BE750
:107E70008093E80098CF2896DEBFCDBFCF91DF91E9
:107E8000FF91EF91BF91AF919F918F917F916F91F2
:107E90005F914F913F912F911F910F91FF90EF9024
:107EA0000F900FBE0F901F901895E0EEF0E08081CC
:107EB0008160808380ED97E00197F1F708958091CC
:107EC000D80080628093D80089B5837E89BD89B54A
:107ED000826089BD09B400FEFDCF8091D8008F7704
:107EE0008093D8008091D80080688093D8008091DA
:107EF000D8008F7D8093D8008091E0008E7F8093A2
:107F0000E00088E08093E2000E94A23D089555279A
:107F1000002480FF02C0060E571F660F771F6115F1
:107F2000710521F096958795009799F7952F802DEB
:067F30000895F894FFCF54
:107F36002A0300000000000000000000000000000E
:107F4600000000000000000000000000000000002B
:107F560000000000000000000000040309041201F4
:107F66000001FE000040B72040150100000001019D
:107F76000902120001010080140904000000FE013C
:107F8600020000640000020009210FFFFF4000010B
:047F960001000000E6
:040000030000700089
:00000001FF
